S0220000687474703A2F2F737265636F72642E736F75726365666F7267652E6E65742F1D
S12300000C9438000C94281A0C9458200C945F000C945F000C945F000C945F000C945F000F
S12300200C945F000C9466230C945F000C94FE260C945F000C947A1A0C94021A0C94D41856
S12300400C94FE270C945F000C947D270C945F000C949D280C9465280C945F000C945F0005
S12300600C945F000C945F000C945F000C945F0011241FBECFEFD0E1DEBFCDBF14BEA895C7
S123008088E10FB6F89480936000109260000FBE15E0A0E0B1E0E4EBF4E502C005900D92BC
S12300A0A832B107D9F717E0A8E2B5E001C01D92A231B107E1F70E947F120C94592A0C94FB
S12300C0000020E030E0D901AC54BF4F0E943B2A802DF901ED5BFE4F80832F5F3F4F203A68
S12300E0310589F720E030E0D901A857BE4F0E943B2A802DF901E45CFE4F80832F5F3F4FF6
S12301002530310589F712BC11BC089520E030E0F901ED5BFE4F8081D901AC54BF4F082EDA
S12301200E94482A2F5F3F4F203A310589F712BC11BC0895199B11C020E030E0D9015096EE
S12301400E943B2A802DF901ED51FE4F80832F5F3F4F203A310591F0F1CF20E030E0D90188
S1230160A859BD4F0E943B2A802DF901ED51FE4F80832F5F3F4F203A310589F712BC11BC6B
S12301800895199B11C020E030E0F901ED51FE4F8081D9015096082E0E94482A2F5F3F4F7D
S12301A0203A310591F0F1CF20E030E0F901ED51FE4F8081D901A859BD4F082E0E94482AA3
S12301C02F5F3F4F203A310589F712BC11BC089520E931E0D9010E943B2A802D2055314029
S12301E0F901ED57FD4F80832F5A3E4F81E0203F380781F712BC11BC089520E430E0F9019B
S1230200ED57FD4F8081D901A05BBE4F082E0E94482A2F5F3F4F203A310589F712BC11BC56
S12302200895A2E0B0E00E943B2A802D90E090931E0180931D0120911D0130911E01A3E042
S1230240B0E00E943B2A802D90E0982F8827820F931F90931E0180931D01ADEEB3E00E94EA
S12302603B2A802D90E090932201809321012091210130912201AEEEB3E00E943B2A802DE3
S123028090E0982F8827820F931F909322018093210180911D0190911E01909320018093F0
S12302A01F01A4E0B0E00E943B2A802D90E090932401809323012091230130912401A5E023
S12302C0B0E00E943B2A802D90E0982F8827820F931F9093240180932301A6E0B0E00E9476
S12302E03B2A802D90E090930101809300012091000130910101A7E0B0E00E943B2A802DFF
S123030090E0982F8827820F931F9093010180930001A1E0B0E00E943B2A802D8093280572
S1230320A8E0B0E00E943B2A802D80931301A9E5B1E00E943B2A802D80932D01A2E0B4E09C
S12303400E943B2A902D892F8150843078F080912D01843039F481E08093180183E6809307
S1230360FB0506C082E08093180102C090931801A9E0B0E00E943B2A802D80931201AEE0A6
S1230380B0E00E943B2A802D80932601ABE0B0E00E943B2A802D80931901A3E0B4E00E9426
S12303A03B2A802D80931A01ACE0B0E00E943B2A802D80931B01AFE6B1E00E943B2A802D20
S12303C080931C01A2EFB1E00E943B2A802D80939C0580919C05882319F081E080939C05E4
S12303E0ADE0B0E00E943B2A802D26E0829FC00111249093150180931401A1E7B1E00E94EF
S12304003B2A802D80931F06A0E7B1E00E943B2A802D80931D068AE080934C0681E0809349
S12304204A06AFE8B1E00E943B2A802D80932E0180912E0181FF05C080912E01827F809371
S12304402E0180912E0185FF05C080912E018F7280932E01A4EFB1E00E943B2A802D90E015
S12304602CE231E0AC01429FC001439F900D529F900D11249093F6058093F505A5EFB1E078
S12304800E943B2A802D8093F205A6EFB1E00E943B2A802D8093F005A7EFB1E00E943B2A8A
S12304A0802D8093EF05A8EFB1E00E943B2A802D90E09093EE058093ED052091ED053091B9
S12304C0EE05A9EFB1E00E943B2A802D90E0982F8827820F931F9093EE058093ED05ABEF6A
S12304E0B1E00E943B2A802D90E09093300180932F0120912F0130913001ACEFB1E00E940B
S12305003B2A802D90E0982F8827820F931F9093300180932F01ADEFB1E00E943B2A802D24
S123052090E090933201809331012091310130913201AEEFB1E00E943B2A802D90E0982FBC
S12305408827820F931F9093320180933101AFEFB1E00E943B2A802D90E09093B6048093C7
S1230560B5042091B5043091B604A0E0B2E00E943B2A802D90E0982F8827820F931F9093C7
S1230580B6048093B50420E030E0D901A25ABE4F0E943B2A802DF901ED5DFC4F8083D901BE
S12305A0AE58BE4F0E943B2A802DF901E450FA4F8083D901A458BE4F0E943B2A802D808B54
S12305C02F5F3F4F2A30310501F7A7E0B2E00E943B2A802D80933701A3E0B2E00E943B2A3F
S12305E0802D8093380120E030E0F901E75DF94F84E6808BD901A45EBD4F0E943B2A802D57
S123060080832F5F3F4F2031310579F720E030E0D901A759BE4F0E943B2A802DF901E85DD6
S1230620FE4F80832F5F3F4F2430310589F720E030E0D901A25DBD4F0E943B2A802DF9019D
S1230640E650FB4F80832F5F3F4F2031310589F7ADE6B1E00E943B2A802D80932501A1EF4F
S1230660B1E00E943B2A802D80939B05A0EFB1E00E943B2A802D80932C01A6E0B2E00E94B0
S12306803B2A802D8093270120E030E0D901AA54BC4F0E943B2A802DF901E35DFC4F8083DA
S12306A02F5F3F4F2031310589F7A7ECB3E00E943B2A802D80933A01A8ECB3E00E943B2ABD
S12306C0802D80933B01A4EDB3E00E943B2A802D8093A705A5EDB3E00E943B2A802D809397
S12306E0A805A6EDB3E00E943B2A802D8093A905A7EDB3E00E943B2A802D8093AA05A8ED7C
S1230700B3E00E943B2A802D8093AB05A9EDB3E00E943B2A802D8093AC05AAEDB3E00E945E
S12307203B2A802D8093AD05ABEDB3E00E943B2A802D8093AE05A8EEB3E00E943B2A802D5C
S123074090E090933401809333012091330130913401A9EEB3E00E943B2A802D90E0982F96
S12307608827820F931F9093340180933301AAEEB3E00E943B2A802D80939E05ACECB3E024
S12307800E943B2A802D2AE0829FC00111249093B6058093B505A1EDB3E00E943B2A802D00
S12307A0829FC00111249093BB058093BA05A2EDB3E00E943B2A802D829FC0011124909359
S12307C0BD058093BC0512BC11BC089580911D0190911E01A2E0B0E0082E0E94482A80916B
S12307E01D0190911E01892F9927A3E0B0E0082E0E94482A8091230190912401A4E0B0E033
S1230800082E0E94482A8091230190912401892F9927A5E0B0E0082E0E94482A8091000126
S123082090910101A6E0B0E0082E0E94482A8091000190910101892F9927A7E0B0E0082E37
S12308400E94482A80911301A8E0B0E0082E0E94482A80911201A9E0B0E0082E0E94482A72
S123086012BC11BC089580E0A1EFB1E0082E0E94482A8AE0A0EFB1E0082E0E94482A80918C
S12308809C05A2EFB1E0082E0E94482A84E0A9E5B1E0082E0E94482A85E0ACE0B0E0082EC3
S12308A00E94482A82E3AFE6B1E0082E0E94482A24E1A1E7B1E0022E0E94482A91E0A0E7F1
S12308C0B1E0092E0E94482A88ECA4EFB1E0082E0E94482AA5EFB1E0092E0E94482AA6EF51
S12308E0B1E0022E0E94482A8AE5A7EFB1E0082E0E94482A88EEA8EFB1E0082E0E94482A57
S123090083E0A9EFB1E0082E0E94482A80912F0190913001ABEFB1E0082E0E94482A8091E4
S12309202F0190913001892F9927ACEFB1E0082E0E94482A8091310190913201ADEFB1E07F
S1230940082E0E94482A8091310190913201892F9927AEEFB1E0082E0E94482A8091B504F8
S12309609091B604AFEFB1E0082E0E94482A8091B5049091B604892F9927A0E0B2E0082EBA
S12309800E94482A8CEDA7E0B2E0082E0E94482A86EEA3E0B2E0082E0E94482A2CE132E071
S12309A088ECD901082E0E94482A2F5F3F4F82E02C323807A9F782E2AFE8B1E0082E0E947C
S12309C0482A81E0A6E0B2E0082E0E94482A12BC11BC0895CF92DF92EF92FF920F931F936E
S12309E0CF93DF93C0E0D0E0A5E0B2E00E943B2A202D30E040E050E0A3EDB3E00E943B2ADA
S1230A00602D6E01CC0CDD1C8DE393E0C80ED91EF601E080F18070E080E090E00E94AC29F6
S1230A2000E010E0A80197010E94AC2924E630E040E050E00E94FE2979018A01CA01B9016D
S1230A4024EF31E040E050E00E94AC2928EC30E040E050E0E20EF31E041F151FA80197019A
S1230A600E94FE29CA01B9012FEF30E040E050E00E94AC2925E030E040E050E00E94FE2901
S1230A80E2E0220F331F441F551FEA95D1F7CA01B90124E630E040E050E00E94FE29F60140
S1230AA0318320832196C732D10509F09DCFC0E0D0E0A9ECB3E00E943B2A202D30E040E0F4
S1230AC050E0A3EDB3E00E943B2A602D6E01CC0CDD1C8BE893E0C80ED91EF601E080F18070
S1230AE070E080E090E00E94AC2900E010E0A80197010E94AC2924E630E040E050E00E94C7
S1230B00FE2979018A01CA01B90124EF31E040E050E00E94AC2928EC30E040E050E0E20ED1
S1230B20F31E041F151FA80197010E94FE29CA01B9012FEF30E040E050E00E94AC2925E0C0
S1230B4030E040E050E00E94FE2992E0220F331F441F551F9A95D1F7CA01B90124E630E006
S1230B6040E050E00E94FE29F601318320832196C732D10509F09DCFC0E0D0E0AAECB3E0A6
S1230B800E943B2A202D30E040E050E0A3EDB3E00E943B2A602D6E01CC0CDD1C89ED93E0BD
S1230BA0C80ED91EF601E080F18070E080E090E00E94AC2900E010E0A80197010E94AC297D
S1230BC024E630E040E050E00E94FE2979018A01CA01B90124EF31E040E050E00E94AC2969
S1230BE028EC30E040E050E0E20EF31E041F151FA80197010E94FE29CA01B9012FEF30E068
S1230C0040E050E00E94AC2925E030E040E050E00E94FE2902E0220F331F441F551F0A9500
S1230C20D1F7CA01B90124E630E040E050E00E94FE29F601318320832196C732D10509F063
S1230C409DCFC0E0D0E0A4E0B2E00E943B2A202D30E040E050E0A3EDB3E00E943B2A602D53
S1230C606E01CC0CDD1C87E294E0C80ED91EF601E080F18070E080E090E00E94AC2900E047
S1230C8010E0A80197010E94AC2924E630E040E050E00E94FE2979018A01CA01B90124EFD8
S1230CA031E040E050E00E94AC2928EC30E040E050E0E20EF31E041F151FA80197010E94A9
S1230CC0FE29CA01B9012FEF30E040E050E00E94AC2925E030E040E050E00E94FE29B2E0AF
S1230CE0220F331F441F551FBA95D1F7CA01B90124E630E040E050E00E94FE29F60131831C
S1230D0020832196C732D10509F09DCFDF91CF911F910F91FF90EF90DF90CF900895EAE7D7
S1230D20F0E0108280E280937C0080E880BF87EE808311B808950F931F93CF93DF93282F58
S1230D4030E0F901EE0FFF1FEE5FFE4F0081118143E0033F140718F0E2E3F0E04CC053E061
S1230D600F3D150718F0EAE0F0E045C0C0E0D0E087E290E0A901489F9001499F300D589FF9
S1230D80300D1124D901AC0FBD1FAA0FBB1FA35CBC4F8D919C9111978017910730F5FE0189
S1230DA03197E20FF31FEE0FFF1FE35CFC4F20813181608171814D915C91FE01EE0FFF1FB4
S1230DC0EE0FFF1FEC0FFD1F3596201B310BC901880F991F880F991F641B750B820F931FF1
S1230DE00E94D729E60FF71F06C02196C732D10549F6E8ECF0E0CF01DF91CF911F910F9123
S1230E0008950F931F93CF93DF93AC01E0E0F0E0EF01CC0FDD1FDE01AB58BB4F8D919C91CE
S1230E20119748175907C0F56D917C913197EE0FFF1FDF01AB58BB4F8D919C911197681B41
S1230E40790B8D919C91C357DB4F28813981E357FB4F00811181481B590B84E690E0DC0103
S1230E604A9FC0014B9F900D5A9F900D11240E94D729201B310B0190F081E02D629FC00188
S1230E80639F900D729F900D112464E670E00E94D7296E0F7F1F09C03196EA30F10509F0DC
S1230EA0B7CF6091A1047091A204CB01DF91CF911F910F91089580912A0590912B05282FFA
S1230EC0205527FF0AC08091140190911501BC01660F771F680F791F1EC02F312CF060912A
S1230EE014017091150117C04091140150911501332727FD309588E290E0821B930B9C0119
S1230F00249FC001259F900D349F900D11246AE070E00E94D729CB0108950F931F93CF93E8
S1230F20DF93AC018091B8049091B9044817590718F4E0EFF0E057C08091D4049091D5047F
S1230F408417950718F4E0E0F0E04DC0E1E0F0E0EF01CC0FDD1FDE01A854BB4F8D919C9125
S1230F60119748175907C0F56D917C913197EE0FFF1FDF01A854BB4F8D919C911197681B07
S1230F80790B8D919C91EA52FB4F20813181CA52DB4F08811981481B590B84E690E0DC01BE
S1230FA04A9FC0014B9F900D5A9F900D11240E94D729201B310B0190F081E02D629FC00147
S1230FC0639F900D729F900D112464E670E00E94D729E61BF70B07C03196EE30F10509F0B1
S1230FE0B7CFEEEFF0E0CF01DF91CF911F910F9108958091B305882359F08CED95E090935F
S12310003601809335011092C8051092C7052AC08091B305882349F08CED95E09093360190
S12310208093350184E690E019C08091B305882349F08CED95E090933601809335018AEFF9
S123104090E00CC08091B305882361F08CED95E0909336018093350184EF91E09093C80526
S12310608093C705F89480919705909198058A5A9A4AC1F0809197059091980585559545FE
S123108089F0789480912706909128068064909328068093270684EF91E090933601809374
S12310A035010AC0789480912706909128068F7B9093280680932706F8948091990590919C
S12310C09A058F3F89F0789480912706909128068068909328068093270684EF91E090930D
S12310E03601809335010AC0789480912706909128068F779093280680932706809135012B
S123110090913601892B99F12F9A2091C7053091C8052115310511F42F9A16C08091C50576
S12311209091C605029780F485B1881F8827881F809587958827879595B19F77982B95B916
S12311403093C6052093C5058091C5059091C60501979093C6058093C505809135019091EE
S123116036010197909336018093350108952F981092C8051092C7050895809127069091BC
S123118028069F779093280680932706809100019091010197FD44C08091280580FF32C0FA
S12311A020918F053091900580911F01909120018C599F4F8217930720F461E070E040E84A
S12311C032C020918F053091900580911F019091200149978217930720F461E070E048E02B
S12311E022C020918F053091900580911F0190912001845690408217930790F461E070E009
S123120044E011C020918F053091900580911F01909120018217930718F460E070E802C02E
S123122060E070E040E02091270630912806CB019927869597958827822B932B90932806EF
S1231240809327062091270630912806CB0180709078822B932B90932806809327068091AC
S123126000019091010192FF33C020918F053091900580912F01909130018217930740F52C
S123128020918F0530919005809131019091320128173907E8F420913605309137058091C3
S12312A0250190E001962817390794F48091270690912806946090932806809327068091D3
S12312C0280580FF03C0616048600BC0706809C080912706909128069B7F909328068093BB
S12312E0270620913805309139058091380190E08217930734F480913801882311F0606104
S123130048608091A80520913A0530913B0590E08F5B9F4F8217930774F48091A805882326
S123132051F0606280918F0590919005895B9B40A0F0446012C08091A80520913A05309117
S12313403B0590E0C296821793073CF48091A805882319F0606251E001C050E08091A7050B
S1231360209140053091410590E0C296821793076CF48091A705882349F0606480918F0507
S123138090919005855C994008F044608091A90520913E0530913F0590E0C296821793078A
S12313A034F48091A905882311F0606844608091AA0520913C0530913D0590E0C296821714
S12313C0930734F48091AA05882311F0606844608091AB05209142053091430590E0880FA6
S12313E0991F8217930734F48091AB05882311F0606844608091AC05209144053091450536
S123140090E0880F991F8217930734F48091AC05882311F0606844608091AD052091460515
S12314203091470590E0880F991F8217930734F48091AD05882311F0606844608091AE05E2
S1231440209148053091490590E0880F991F8217930734F48091AE05882311F06068446085
S1231460552321F082E380938B0502C010928B05189B06C060FD02C077FF09C06170707853
S12314807093B1056093B0054093B20506C01092B1051092B0051092B2054093B305089567
S12314A0809100019091010193FF1FC11A9B06C08091B9058F5F8093B90502C01092B90556
S12314C08091B905853108F454C01092B40520918F05309190058091B5049091B60482173F
S12314E0930778F48091B0059091B10582609093B1058093B0058091B20588608093B20548
S123150009C08091B0059091B1058D7F9093B1058093B0058091280583FF16C080918F0579
S123152090919005815D974078F08091B0059091B10584609093B1058093B0058091B205EA
S123154082608093B20509C08091B0059091B1058B7F9093B1058093B0058091B5059091DE
S1231560B6059093B8058093B70584E38093B905B1C08091B7059091B805892B09F45DC0DB
S12315808091B7059091B80501979093B8058093B7058091B405823099F0833030F48823CE
S12315A051F0813009F096C019C08330A9F1843009F090C031C01092B8051092B7058AC0CB
S12315C08091B0059091B10584609093B1058093B0058091B20582608093B20520918F052C
S12315E0309190058091B5049091B6048217930768F48091B0059091B10582609093B10505
S12316008093B0058091B205886059C08091B0059091B1058D7F0CC09091CE058091B70400
S1231620891708F440C08091B0059091B1058B7F9093B1058093B0054DC04E9B20C08091DB
S12316408F05909190058D5D9540C8F08091C3059091C40501969093C4058093C3052091F3
S1231660BA053091BB0528173907A0F58091BC059091BD059093C2058093C10514C0209115
S1231680C1053091C20521153105E1F080918F05909190058D5D9540A8F021503040309365
S12316A0C2052093C1058091B0059091B10584609093B1058093B0058091B2058260809307
S12316C0B20508C01092C4051092C3051092C2051092C1058091B20581FF07C080912E0192
S12316E080FF03C084E68093F10508959C018091280584FF1BC022533040C901F3E0880F42
S1231700991FFA95E1F7220F331F280F391F2455354F442737FD4095542F60E579E784E097
S123172090E00E94202A822F90E008958091280585FD03C084E690E0089522533040C901E2
S123174073E0880F991F7A95E1F7220F331F280F391F2455354F442737FD4095542F60E5B1
S123176079E784E090E00E94202A2C592695822F90E00895A89582E50E94F22883E10E94E1
S1231780F22880918F0590919005892F99270E94F22880918F05909190050E94F228809174
S12317A04005909141050E94F2288091CE050E94F22880912A0590912B050E94F2288091BF
S12317C03805909139050E94F22880913605909137050E94F22880913205909133050E9405
S12317E0F22880919505909196056091180170E00E94D729CB010E94F228809194050E9494
S1231800F228809193050E94F22820912706309128068091F7059091F805E3E09695879543
S1231820EA95E1F78170232F3327822B0E94F22880912706909128060E94F22880916E0679
S123184080950E94F228809149060E94F22880913005909131050E94F2288091F90590910E
S1231860FA05969587950E94F22880917106909172069093430580934205809151069091F3
S1231880520690934505809344052091CB0530E0220F331FF901E65CFA4F80819181892FBF
S12318A0990F990BB3E0220F331FBA95E1F7822B0E94F228E091CB05F0E0EE0FFF1FE65CC4
S12318C0FA4F808191810E94F2288DEA0E94F2288091CB058F5F8093CB05883010F01092AD
S12318E0CB050895CF92DF92EF92FF920F931F93CF93DF93A89588E10FB6F8948093600001
S1231900109260000FBE0E943E29882309F4EDC50E94CF289093CA058093C90581369105D8
S123192009F486C08236910508F041C08D34910509F4E1C18E349105E8F48134910509F4A7
S12319409CC08234910568F48932910509F409C58433910509F4B0C58832910509F0C3C5D3
S1231960DDC48534910509F4C1C08634910509F0BAC545C18335910509F445C58435910583
S123198048F48035910509F48BC38235910509F0AAC502C48735910509F4F9C38835910598
S12319A009F48AC48535910509F09DC53DC48936910509F426C38A369105E8F4843691056F
S12319C009F4A2C28536910548F48236910509F495C28336910509F086C593C28636910539
S12319E009F4EBC08636910508F4F8C18736910509F079C52DC38037910509F456C381379F
S1231A00910548F48D36910509F434C18F36910509F069C569C48937910509F4C5C48A3759
S1231A20910509F4C9C28837910509F05CC5C4C281E60E94F22880EA0E94F2281092CA05D5
S1231A401092C9050EC0ED5BFE4F80810E94F2288091C9059091CA0501969093CA05809387
S1231A60C905E091C905F091CA05E03AF10558F382E30E9443288EE936C51092CA051092B3
S1231A80C905C0E0D0E00E943E29882341F1C091C905D091CA05C03AD10589F40E94CF2809
S1231AA09093CA058093C9058E3B910519F4C6E1DAEF15C08091C9050E94F228FBCF0E9497
S1231AC0CF28CD5BDE4F88838091C9059091CA0501969093CA058093C905C0E0D0E021966B
S1231AE04AEFC030D40708F000C5CDCFC0E0D0E00E943E29882309F459C00E94CF288A3B0D
S1231B00910509F0F2C488E10FB6F89480936000109260000FBE1092CA051092C9053EC0A1
S1231B20885B0E94F2288DEF0E94F2282091C9053091CA058AEF90E0289FE001299FD00D85
S1231B40389FD00D112407C0DE010E943B2A802D0E94F22821962091C9053091CA052F5F2E
S1231B603F4F8AEF90E0AC01249FC001259F900D349F900D112421503040C817D90720F300
S1231B80822F885B80950E94F2288091C9059091CA0501969093CA058093C9058091C905C4
S1231BA09091CA058430910508F4BACF21965AEFC030D50708F099C49BCF86E60E94F228AF
S1231BC080EA0E94F2281092CA051092C9050EC0ED51FE4F80810E94F2288091C9059091E4
S1231BE0CA0501969093CA058093C905E091C905F091CA05E03AF10558F389E974C4109272
S1231C00CA051092C90500E010E00E943E29882349F1C091C905D091CA05C03AD10591F41F
S1231C200E94CF289093CA058093C905893B910519F406E11AEF16C0E091BF05F091C0058C
S1231C40099510C00E94CF28CD51DE4F88838091C9059091CA0501969093CA058093C905EA
S1231C6000E010E00F5F1F4F8AEF0030180708F03CC4CBCF8DE60E94F22889E00E94F22806
S1231C8080911D0190911E010E94F22880911D0190911E01892F99270E94F228809123013D
S1231CA0909124010E94F2288091230190912401892F99270E94F22880910001909101013A
S1231CC00E94F2288091000190910101892F99270E94F228809113010E94F22880911201D6
S1231CE00E94F228AAE0B0E00E943B2A802D0E94F22882E9F8C31092CA051092C905C0E0F3
S1231D00D0E00E943E298A3008F461C00E94CF2890931E0180931D0100911D0110911E01B4
S1231D200E94CF28982F8827800F911F90931E0180931D010E94CF289093240180932301C6
S1231D4000912301109124010E94CF28982F8827800F911F90932401809323010E94CF289E
S1231D60909301018093000100910001109101010E94CF28982F8827800F911F909301017E
S1231D80809300010E94CF28809313010E94CF28809312010E94CF28AAE0B0E0082E0E9421
S1231DA0482A0E941B230E94CF28823B910551F40E94E603E091BF05F091C0050995CFE643
S1231DC0DAEF05C0E091BF05F091C005099521964AEFC030D40708F088C393CF85E60E94EB
S1231DE0F22883E10E94F2281092CA051092C9050EC0ED5DFC4F80810E94F2288091C905C5
S1231E009091CA0501969093CA058093C905E091C905F091CA05EA30F10558F3809119014F
S1231E200E94F22880911B010E94F22883E00E944428809128010E94F228809129010E94B5
S1231E40F22880912A010E94F22880912B010E94F228809114019091150166E070E00E94DE
S1231E60D729CB010E94F228809125010E94F228AEE6B1E00E943B2A802D0E94F2288AE9DB
S1231E800E94F2288CE60E94F22884E10E94F2281092CA051092C9050EC0E450FA4F808106
S1231EA00E94F2288091C9059091CA0501969093CA058093C905E091C905F091CA05EA3080
S1231EC0F10558F31092CA051092C9050EC0E450FA4F80890E94F2288091C9059091CA05FD
S1231EE001969093CA058093C905E091C905F091CA05EA30F10558F383E9F5C20E9486003F
S1231F00F4C20E94C100F1C281E50E94F22880E10E94F2288091F6049091F7040E94F228CF
S1231F2080915806909159060E94F22880915A0690915B060E94F22880915C0690915D064C
S1231F400E94F22880915E0690915F060E94F22880916006909161060E94F22880916206D6
S1231F60909163060E94F22880913205909133050E94F2288091B2050E94F2288091B00570
S1231F809091B1050E94F22880916E0680950E94F2288091CE050E94F22880911C060E94DF
S1231FA0F22884E00E94F22885E00E94F22886E00E94F2288EEA97C20E94BA0B96C20E946E
S1231FC0CF28C82FD0E00E94CF28C817D90709F08CC20E94CF288C019093CA058093C905C7
S1231FE00E94CF280817190709F07FC20E94CF288639910509F079C28091C905CD5BDE4F75
S12320004DC00E943E298530D0F6FBCF0E94CF28C82FD0E00E94CF28C817D90709F065C2A9
S12320200E94CF288C019093CA058093C9050E94CF280817190709F058C20E94CF2888395E
S1232040910509F052C28091C905CD51DE4F26C00E943E298530D0F6FBCF0E94CF28C82FEB
S1232060D0E00E94CF28C817D90709F03EC20E94CF288C019093CA058093C9050E94CF28C9
S12320800817190709F031C20E94CF288F3A910509F02BC28091C905CD57DD4F888325C212
S12320A00E943E298530C8F6FBCFC0E0D0E00E943E29823080F10E94CF280E94CF288F3861
S12320C0910509F012C21092CA051092C9051CC0ED57FD4F108180E70E94F22882E00E9494
S12320E0F2288091C9050E94F228812F0E94F2288FE80E94F2288091C9059091CA05019622
S12321009093CA058093C905E091C905F091CA05E03AF105E8F221965AEFC030D50709F4A6
S1232120E4C1C5CF0E94CF288C010E94CF28D82FCC27C00FD11F0E94CF288C019093CA05D2
S12321408093C9050E94CF280817190709F0CDC10E94CF28883A9105A9F4DE010E94432ABF
S1232160E0708091C9059091CA05E82BF92BF093CA05E093C905DE010F010E94542A12BC95
S123218011BCB3C1E091BF05F091C00509950E943E29853038F6FBCFCC24DD240E943E2931
S12321A08330C0F10E94CF288C010E94CF28EC010E94CF288D3A910509F097C1FC2EEE2488
S12321C0E00EF11ED7010E943B2A802D90E0D70111960E943B2A002D10E0102F0027080FE2
S12321E0191F84E50E94F22884E00E94F228802F0E94F2288E2D0E94F228EF2CFF248E2D83
S12322000E94F228012F1127802F0E94F2288BEA0E94F2280894C11CD11C80E0C8168AEFDD
S1232220D80609F462C1BACFCC24DD240E943E298330C0F10E94CF288C010E94CF28EC0109
S12322400E94CF288A3A910509F04FC1FC2EEE24E00EF11ED7010E943B2A802D90E0D70171
S123226011960E943B2A002D10E0102F0027080F191F85E50E94F22884E00E94F228802FE5
S12322800E94F228012F1127802F0E94F2288E2D0E94F228EF2CFF248E2D0E94F2288AEA0B
S12322A00E94F2280894C11CD11C40E0C4164AEFD40609F41AC1BACFC0E0D0E00E943E2931
S12322C0882359F00E94CF28873A910509F00DC1E091BF05F091C005099521965AEFC03046
S12322E0D50709F402C1EACFC0E0D0E00E943E29882369F00E94CF288039910509F0F5C092
S12323000E94FD00E091BF05F091C005099521968AEFC030D80709F4E8C0E8CFC0E0D0E056
S12323200E943E298823B1F00E94CF28873D910509F0DBC08091360590913705ADE6B1E0F0
S1232340082E0E94482A12BC11BCE091BF05F091C005099521964AEFC030D40709F4C5C03E
S1232360DFCFC0E0D0E00E943E298823B1F00E94CF28863D910509F0B8C080913605909136
S12323803705AEE6B1E0082E0E94482A12BC11BCE091BF05F091C005099521965AEFC030EA
S12323A0D50709F4A2C0DFCFC0E0D0E00E943E29823010F10E94CF28892B09F096C00E94E6
S12323C0CF2886389105C1F489E70E94F22885E00E94F2288FEC0E94F2288FE30E94F22847
S12323E08DE00E94F22885E40E94F2288CE00E94F22886E80E94F22821968AEFC030D8073A
S123240009F473C0D3CFC0E0D0E00E943E29823008F44CC00E94CF28892B09F047C00E94E4
S1232420CF288C3A910509F060C083E50E94F22888E00E94F22880919705909198050E94D7
S1232440F2288091970590919805892F99270E94F22880912506909126060E94F228809169
S1232460250690912606892F99270E94F22880912006909121060E94F22880912006909119
S12324802106892F99270E94F22880917406909175060E94F2288091740690917506892F1B
S12324A099270E94F2288CEA0E94F22821964AEFC030D407D1F0A9CFC0E0D0E00E943E291D
S12324C0823058F00E94CF28892B79F40E94CF288B3C910511F40E94110121965AEFC030A5
S12324E0D50719F0EBCF0E94F228A895DF91CF911F910F91FF90EF90DF90CF9008950F9305
S12325001F93CF93DF9310922806109227060E943B283D9A3E9A3C9A459A469A449A3F9A92
S1232520479A38984098399841983A9842983B984398389839983A983B9854985C985598F7
S12325405D9854985598239A269A279A2B9A2E982F98259A249A5398529822985698219866
S123256020980E944628AAE5B1E00E943B2A802D80939D050E94C6220E941B230E942928A9
S12325800E948F060E94EA042B9A2E98A7E0B0E00E943B2A802D12BC11BC85FF9BC080918F
S12325A00001909101019F7D90930101809300010E94E6030E9433040E94C1000E948600AF
S12325C00E94FD0086E0AAE0B0E0082E0E94482A89E1ABE0B0E0082E0E94482A8EE1ACE0C4
S12325E0B0E0082E0E94482AAEE0B0E0082E0E94482A20E030E0F901ED5DFC4F8081D9011B
S1232600A25ABE4F082E0E94482A2F5F3F4F2A30310589F780912801A9E6B1E0082E0E9405
S1232620482A80912901AAE6B1E0082E0E94482A80912A01ABE6B1E0082E0E94482A8091C5
S12326402B01ACE6B1E0082E0E94482A20E030E0F901E450FA4F8081D901AE58BE4F082E32
S12326600E94482A2F5F3F4F2A30310589F720E030E0F901E450FA4F8089D901A458BE4FA3
S1232680082E0E94482A2F5F3F4F2A30310589F780911F06A1E7B1E0082E0E94482A809116
S12326A014019091150166E070E00E94D729ADE0B0E0062E0E94482A84E1ADE6B1E0082E6E
S12326C00E94482A81EEAEE6B1E0082E0E94482A12BC11BC0E94E8000E9411010E949A00EF
S12326E00E946100809100019091010185FD07C080916F008B7F80936F00459A469A809179
S12327002701882311F480E801C080E4809339011092290580911401909115018D5A9D4012
S123272030F08CEA9DE0909315018093140110928C0586B3866086BB78948AEA0E94F22852
S123274080E00E94F22885E50E94F22883B18695817080939F0580916E00836080936E0059
S12327602B9A2E9AA89580918F05909190058635910570F180918C05882351F580912706AD
S1232780909128069F7E909328068093270680916F00856080936F0080916E0083608093DC
S12327A06E002B9A81E080938C05809127069091280680629093280680932706809127069F
S12327C0909128069062909328068093270649C080918C05813009F044C080918F05909104
S12327E090058234910508F03CC080916F008D7F80936F00809170008C7F809370008091D2
S12328006F008B7F80936F0080916E00836080936E0080912706909128068F7D90932806EC
S1232820809327068091270690912806877F9093280680932706389839983A983B985498FE
S12328405598459A469A449A10928C0580912706909128069F7D90932806809327061092DB
S12328608A0580918C058130D9F480916F00826080936F00809170008360809370008091C9
S12328806E00836080936E008091270690912806886090932806809327062B9A2E9A14C0FB
S12328A010928A05459A469A449A10928A051092B3001092960510929505809141019091D3
S12328C04201892B09F42B9880912905833009F4DCC0843018F4882371F077C0853009F4FD
S12328E0E7C1853008F442C1863009F4CDC1873009F093C21CC280918D0590918E05853642
S1232900910508F48DC2E0912905F0E080917800909179008C7F65E070E00E94D729EE0F01
S1232920FF1FE659FA4F7183608380912905C82FD0E0E0912905F0E0EE0FFF1FE65DFA4F1A
S123294080819181E0912905F0E0EE0FFF1FE659FA4F20813181880F991F880F991F820FCC
S1232960931F880F991F6AE070E00E94D729CC0FDD1FC65DDA4F7983688310928E05109235
S12329808D05809129058F5F8093290580912905806480937C000E94720C0E945B0790933A
S12329A01701809316018091410190914201892B09F431C280914101909142010197909304
S12329C04201809341012B9A26C280918D0590918E058536910508F423C290912905409105
S12329E0AF05842F83708450990F990F980FE92FF0E0EE0FFF1FEE5FFE4F8081918120914D
S1232A00780030917900820F931F969587959183808310928E0510928D05A895809129057A
S1232A20C42FD0E08130D1F48E01085F1F4F842F0E949B06000F111F065D1A4FF801918307
S1232A4080838091AF058823A9F480913A0590913B050E94760B80934D060CC08081918149
S1232A6062E070E00E94EB29CC0FDD1FCE5BDA4F79836883809129058F5F8093290580917B
S1232A802905806480937C00CBC180918D0590918E058536910508F4C3C1E0912905F0E06E
S1232AA080917800909179009695879596958795EE0FFF1FE659FA4F918380838091290568
S1232AC0C82FD0E0E0912905F0E0EE0FFF1FE65DFA4F80819181E0912905F0E0EE0FFF1F98
S1232AE0E659FA4F20813181880F991F880F991F820F931F880F991F6AE070E00E94D7298B
S1232B00CC0FDD1FC65DDA4F7983688310928E0510928D05809129058F5F809329058091BF
S1232B20290590913901892B80937C000E94720CA8958091AF058F5F8093AF05843010F03A
S1232B401092AF052091AF05922F91709295990F907E85B18F7D892B85B9220F220F220F50
S1232B60207185B18F7E822B85B95AC180918D0590918E058159914008F452C1809127012D
S1232B80882329F1E0912905F0E080917800909179009695879596958795EE0FFF1FE659F2
S1232BA0FA4F91838083A0912905B0E0E0912905F0E0EE0FFF1FE659FA4F80819181AA0FE4
S1232BC0BB1FA65DBA4F11969C938E933EC0E0912905F0E08091780090917900EE0FFF1F69
S1232BE0E659FA4F9183808380912905C82FD0E0E0912905F0E0EE0FFF1FE65DFA4F0081B5
S1232C001181E0912905F0E0EE0FFF1FE659FA4F808191810E948D079C01220F331F280F6C
S1232C20391FC80143E0880F991F4A95E1F7801B910B820F931F6AE070E00E94D729CC0FB5
S1232C40DD1FC65DDA4F7983688310928E0510928D05809129058F5F80932905809129052B
S1232C60806880937C0020919F0583B18695817030E090E02817390709F4CDC0E091BF0586
S1232C80F091C0050995C7C080918D0590918E058536910508F4C4C0E0912905F0E080911D
S1232CA078009091790096958795969587950FC080918D0590918E05893C910508F4B0C083
S1232CC0E0912905F0E08091780090917900EE0FFF1FE659FA4F91838083A0912905B0E0B5
S1232CE0E0912905F0E0EE0FFF1FE65DFA4F20813181E0912905F0E0EE0FFF1FE659FA4F55
S1232D0080819181820F931F96958795AA0FBB1FA65DBA4F11969C938E9310928E051092A5
S1232D208D05809129058F5F809329056DC080918D0590918E058536910508F471C0E0911C
S1232D402905F0E08091780090917900969587959695879590E0EE0FFF1FE659FA4F918399
S1232D608083E0912905F0E0EE0FFF1FE65DFA4F80819181843691050CF5A0912905B0E0E3
S1232D80E0912905F0E0EE0FFF1FE65DFA4F40815181E0912905F0E0EE0FFF1FE659FA4F74
S1232DA020813181CA01880F991F840F951F820F931F969587959695879519C0A091290552
S1232DC0B0E0E0912905F0E0EE0FFF1FE65DFA4F20813181E0912905F0E0EE0FFF1FE6592D
S1232DE0FA4F80819181820F931F96958795AA0FBB1FA65DBA4F11969C938E9310928E051E
S1232E0010928D051092290580912905806480937C000E94720CA89503C081E08093290536
S1232E2080918D0590918E05019690938E0580938D0580918F05909190058752924008F443
S1232E4052C080917A0687FF02C0E0E002C0E0917A0680914B068F5F80934B0690914B06EA
S1232E6080914C06981708F441C010924B0620913805309139054E2F50E0FA01E75DF94F2B
S1232E80808190E02817390754F480914906843634F48091490690914A06890F13C02091C7
S1232EA0380530913905FA01E75DF94F808190E0281739074CF08091490682302CF08091E0
S1232EC0490681508093490620914906FA01E75DF94F8089332727FD309590E082179307F6
S1232EE02CF4808901C081E08093490680918F05909190058739910508F46DC0209136055B
S1232F00309137058091250190E04996281739070CF061C08091F3059091F40501969093B1
S1232F20F4058093F3052091F3053091F4058091F5059091F6052817390708F440C01092E2
S1232F40F4051092F30520918F05309190058091ED059091EE050A972817390730F49091C3
S1232F60F1058091F205890F15C020918F05309190058091ED059091EE054996821793071E
S1232F8058F49091F1058091F005891728F48091F10581508093F1059091F1058091EF050B
S1232FA0891718F48091EF0508C09091F1058091F005981720F48091F0058093F105809194
S1232FC08F05909190058A58924038F48091EF058093F10502C01092F1058091280582FF9C
S1232FE04FC080918F0590919005855F914008F447C080918F0590919005805D974008F0A4
S12330003FC020913605309137058091250190E0059628173907A4F5209136053091370581
S12330208091A20590E00196821793074CF18091A3059091A405A091A505B091A60501967C
S1233040A11DB11D8093A3059093A405A093A505B093A6058091A3059091A405A091A50530
S1233060B091A6058158994AA340B04010F181E08093A1058091270690912806916015C063
S123308080913605909137058093A2051092A3051092A4051092A5051092A6051092A10553
S12330A080912706909128069E7F90932806809327060E94BD080E94500A0E94F9078091BB
S12330C000019091010180FF67C080912E0180FF11C08091EC05883C28F08091F105882302
S12330E0B9F418C09091F1058091EC058695891790F010C080912E0182FF0DC08091EC0593
S1233100883C48F0809127069091280696FF02C0549A01C0549880912E0184FF16C0809186
S1233120EC05883C28F08091490618165CF12CC0209149068091EC05332727FD3095869597
S123314090E0821793070CF11FC080912E0186FF1CC08091EC05883CC0F020918F053091CF
S1233160900580913301909134018217930760F4209138053091390580919E0590E08217EA
S1233180930714F4559A01C055988091EC05883C28F01092EC0502C0549855988091EC05DE
S12331A08F5F8093EC05DDCA1F920F920FB60F9211248F939F9380917B068F5F80937B061D
S12331C080917B06882309F447C080912706909128069061909328068093270610928C0568
S12331E080912706909128069F7D909328068093270680916F008B7F80936F0080916F0005
S12332008D7F80936F00809170008C7F8093700080916E00836080936E00459A469A449A8D
S123322080912706909128068F7D90932806809327068091270690912806877F909328067C
S123324080932706389839983A983B98549855981092900510928F0578949F918F910F90A3
S12332600FBE0F901F9018952091780630917906809184009091850028173907F0F4809164
S123328054068630A1F48091990590919A05880F991F90939A058093990580919905909184
S12332A09A05816090939A058093990504C010929A051092990581E003C0809154068F5F55
S12332C080935406809184009091850090937906809378060895282F80912706909128068E
S12332E093FD0BC0223031F0233031F0213029F44598089546980895449808951F938091E9
S1233300E405882309F45CC08091E4058130A1F4459A1092E4058091F4049091F50490930C
S123332084068093830680918F05909190058559914198F182E02FC08091E4058230A1F43D
S1233340469A1092E4058091F4049091F50490936D0680936C0680918F0590919005855987
S12333609141D8F083E017C08091E4058330A9F4449A1092E4058091F4049091F50490937C
S12333807D0680937C0680918F05909190058559914118F081E00E946B198091200690911F
S12333A02106892B69F180917606882349F1809120069091210690938B0080938A0020C0B8
S12333C0809176068823E1F010917606113041F010917606123021F010917606133031F45C
S12333E0809176060E946B191093E405809174069091750690938B0080938A0010927606FA
S12334001F9108951F920F920FB60F9211242F933F934F935F936F937F938F939F93AF935C
S1233420BF93EF93FF930E947E192B9A7894FF91EF91BF91AF919F918F917F916F915F9128
S12334404F913F912F910F900FBE0F901F9018951F920F920FB60F9211242F933F934F932E
S12334605F936F937F938F939F93AF93BF93EF93FF938091F4049091F50401969093F50470
S12334808093F4048091280587FF23C08091E5058823F9F02091F4043091F504809151061C
S12334A09091520648E750E0BA01681B790B2617370769F02091F4043091F50480917106AF
S12334C090917206481B590B2417350711F40E947E19FF91EF91BF91AF919F918F917F91D3
S12334E06F915F914F913F912F910F900FBE0F901F9018951F920F920FB60F9211248F93F2
S12335009F93F89480915506882309F486C08091B0059091B10597FD80C0809113018095E4
S123352080936E0680916E0690911C068C59891B80936E069091FB05943029F1953040F430
S1233540923051F19330B8F4913009F058C009C09731C1F1933609F441C09E3009F04FC042
S123356023C080916E068093B20084E08093B100389A83E050C080916E0686BD83E085BD40
S12335803A9A84E048C080916E068093B2009093B1003B9A82E03FC080916E0686BD83E068
S12335A085BD399A81E037C081E08093110580916E068093B20084E08093B100389A3B9AF7
S12335C087E129C081E08093120580916E0686BD83E085BD399A3A9A8EE01DC081E0809338
S12335E0110580916E068093B20084E08093B100389A3B9A3A9A399A9093FB050EC08091EF
S12336006E068093B20084E08093B100389A3B9A3A9A399A83E68093FB0578949F918F911F
S12336200F900FBE0F901F901895CF93DF93EC0180919C05E7E0F0E0E81BF109EE0FFF1FFD
S1233640E65DFA4F8081918120919B05821B282F30E080912C0190E0880F991F880F991F26
S1233660AC01429FC001439F900D529F900D112464E670E00E94D7296436710520F083E6F0
S12336808093770602C060937706809177066AE00E94CB2980935006809150068A302CF050
S12336A089E0809350068093500680918F0590919005885E934008F0ADC010924E068FEFDE
S12336C080937A0680915006992787FD9095E4E0880F991FEA95E1F78093930580918F05C9
S12336E09091900564E670E00E94D72965506093730680918F0590919005845F914060F450
S123370010927306E0917306FF27E7FDF095E45CFE4F808190E09DC0809173068430D9F5AA
S1233720E0919305F0E0ED5BFE4F2081E0917306FF27E7FDF095E45CFE4F6081E0917306A5
S1233740FF27E7FDF095E45CFE4F808190E09093FA058093F905E091F905F091FA058091A5
S12337608F05909190054091730630E0220F331F261B3109845F91406CE94602A00111247C
S1233780840F951FAC01249FC001259F900D349F900D11243AC0E0917306FF27E7FDF09534
S12337A0E35CFE4F6081E0917306FF27E7FDF095E45CFE4F4081E0917306FF27E7FDF09558
S12337C0E45CFE4F808190E09093FA058093F905E091F905F091FA0580918F05909190056A
S12337E02091730670E0641B7109845F91404CE9240290011124820F931F9C01629FC001DB
S1233800639F900D729F900D112464E670E00E94D729BBC080918F0590919005875F924256
S1233820E8F086E980934E068FE080937A068091500690917A068295807F890F8093930573
S1233840E0919305F0E0ED5BFE4F808190E0880F991F9093FA058093F9059DC080918F0501
S123386090919005885E934062E370E00E94D72960934E0680914E066AE00E94CB298093FF
S12338807A068091500690917A068295807F890F80939305E0919305F0E0ED5BFE4F8081D4
S12338A090E0880F991F9093FA058093F90580917A0687FD36C080917A068F3094F5E091BD
S12338C09305F0E0EC5BFE4F6081E0919305F0E0ED5BFE4F5081E091F905F091FA058091C8
S12338E04E0620917A0690E04AE0240290011124821B930B880F991F70E0651B7109AC0138
S1233900469FC001479F900D569F900D11246AE070E00E94EB29E60FF71FF093FA05E09363
S1233920F9058091500687FD36C080915006893094F5E0919305F0E0ED5AFE4F6081E0913C
S12339409305F0E0ED5BFE4F5081E091F905F091FA05809177062091500690E04AE0240251
S123396090011124821B930B880F991F70E0651B71099C01269FC001279F900D369F900DB1
S123398011246AE070E00E94EB29E60FF71FF093FA05E093F9058091270690912806977FFD
S12339A090932806809327068091F7059091F805877F9093F8058093F7058091B20588239F
S12339C009F458C08091B20588233CF18091B205883088F08091530690E083709070892BB5
S12339E009F448C08091530667E00E94CB29992309F440C012C08091B2058430C0F08091AF
S1233A00530690E083709070892B39F08091530667E00E94CB29992369F580912706909149
S1233A2028069860909328068093270623C08091B205823050F08091F7059091F80588601B
S1233A409093F8058093F70515C08091B205882389F08091F9059091FA058739910550F0AD
S1233A608091F9059091FA058C5890409093FA058093F905809153068F5F80935306409197
S1233A80CE05445645310CF044E18091F9059091FA0520911201885B9F4F820F911D6AE0D1
S1233AA070E00E94D729709372066093710680918F0590919005209171063091720668E225
S1233AC070E00E94D729260F311D30935206209351062091F9053091FA0580911201909194
S1233AE08B05285B3F4F280F311D291B3109842F4C3E0CF48CEE992787FD9095280F391F6F
S1233B003093CD052093CC058091CC059091CD058D5B92402CF06CEB72E080E090E015C08F
S1233B208091CC059091CD0505972CF465E070E080E090E00AC08091CC059091CD05AC013F
S1233B40BA01882777FD8095982F20919105309192052C0F3D1F40E050E00E94AC2920EB9F
S1233B6034E040E050E00E94FE29C21BD30BCE01DF91CF910895A0E0B0E0BC01CD0128E575
S1233B8032E040E050E00E94AC2920EB34E040E050E00E94FE29DA01C90108950F931F937A
S1233BA0CF93DF9380910A0590910B05909382068093810680910A0590910B05499708F46A
S1233BC071C280917B06882349F088EE9DEF90930F0580930E0510927B0653C080918F05FE
S1233BE09091900540910E0550910F05895B9B40C0F0E0919105F091920520910A05309123
S1233C000B058091F80490E0241B350BAC01429FC001439F900D529F900D112464E170E06E
S1233C2017C0E0919105F091920520910A0530910B058091F80490E0241B350BAC01429F6F
S1233C40C001439F900D529F900D11246EE170E00E94EB29CB018E0F9F1F62E070E00E94AD
S1233C60EB297093920560939105109292051092910580910A0590910B0590930F058093FD
S1233C800E0580918A05893628F480918A058F5F80938A0580918F0590919005C0910E05A3
S1233CA0D0910F05D0932606C0932506209125063091260600910C0510910D0540E050E010
S1233CC060E070E489E191E00E94202ACA01B90124E130E040E050E00E94AC2920EC30E008
S1233CE0A901049F9001059F300D149F300D11242050324040E050E00E94FE293093900589
S1233D0020938F0580918F05909190058D5D954010F0E8981AC0E89A80918F059091900507
S1233D208C54944090F48091F6049091F7048737910558F08091F6049091F7048A37910506
S1233D4020F481E08093E50502C01092E5052091DB053091DC054091D9055091DA05C90133
S1233D60880F991F820F931F840F951F96958795969587959093DC058093DB058091D705F4
S1233D809091D8059093DA058093D9058091D5059091D6059093D8058093D7058091D3056F
S1233DA09091D4059093D6058093D5058091D1059091D2059093D4058093D3058091CF056F
S1233DC09091D0059093D2058093D10580918F05909190059093D0058093CF0580918F0527
S1233DE0909190058D5D9540B8F08091CE054091CF055091D0052091DB053091DC0590E0C0
S1233E00821B930B840F951F9695879596958795855B8093CE050FC084E68093CE05809198
S1233E2091059091920564E070E00E94EB29709392056093910510927B0680918F059091DA
S1233E4090058C529140A0F580910C0590910D05039771F580915406813051F584E090E0FA
S1233E6090930D0580930C0580910C0590910D0580688093810080918400909185009695AE
S1233E808795969587959093850080938400D695C795D695C795D0930F05C0930E05809100
S1233EA025069091260696958795969587953AC080918F0590919005875B9340B8F1809134
S1233EC00C0590910D05049789F580915406813069F583E090E090930D0580930C058091CA
S1233EE00C0590910D058068809381008091840090918500880F991F880F991F909385007D
S1233F0080938400CC0FDD1FCC0FDD1FD0930F05C0930E058091250690912606880F991FA3
S1233F20880F991F909326068093250680912506909126060E94151B90937506809374061B
S1233F408091F7059091F80583FF3AC0E091E605F091E705CF0183709070892B99F4209138
S1233F6025063091260680912506909126066AE070E00E94D729261B370B309375062093EC
S1233F80740618C020913A01809125069091260668E270E00E94D72930E0629FC001639F46
S1233FA0900D729F900D11248C599F4F90937506809374063196F093E705E093E60504C027
S1233FC01092E7051092E60580918F05909190058A58924038F080912A0590912B058E3636
S1233FE091053CF48CE291E090937F0680937E0604C010927F0610927E068091740690911C
S12340007506209116013091170140917E0650917F06821B930B841B950B90936B068093A4
S12340206A0680916A0690916B0697FF20C080916A0690916B0620912506309126064091D6
S1234040740650917506820F931F8417950778F420912506309126068091740690917506B0
S1234060821B930B449690936B0680936A06F89480915406833011F48EE005C080915406C3
S1234080843081F487E18093FB0580912506909126060E94BB1D909389008093880081E0CD
S12340A0809355067894DF91CF911F910F9108951F920F920FB60F9211242F933F934F9362
S12340C05F936F937F938F939F93AF93BF93EF93FF934B9926C0E0915406F0E08091F4046C
S12340E09091F504EE0FFF1FEA5AF94F918380830E94CE1D0E9434198091970590919805FD
S1234100880F991F9093980580939705809197059091980581609093980580939705479843
S123412022C2209184003091850080910A0590910B05969587952817390770F480918F05FC
S123414090919005815D974038F081E090E0909398058093970507C28091F7059091F80594
S123416083FFA2C0809184009091850090930B0580930A05109285001092840080919705CD
S123418090919805880F991F9093980580939705479A20913A01809125069091260668E2FF
S12341A070E00E94D72930E0629FC001639F900D729F900D11248C599F4F90937506809331
S12341C0740680918F05909190058051974208F057C0809127069091280693FD51C080910E
S12341E074069091750690938B0080938A00209125063091260680912506909126069695DD
S1234200879596958795281B390B309321062093200680915406813021F0809154068430A1
S123422031F4449883E08093E40581E01BC080915406853021F080915406823031F445988E
S123424081E08093E40582E00DC080915406833021F080915406863039F4469882E08093FE
S1234260E40583E0809376068EEB90E0909323068093220680912706909128069F770FC07D
S123428080912506909126068C509E4F90938B0080938A00809127069091280690689093D5
S12342A02806809327065FC18091280587FF5CC08091E505882309F457C08091F4049091A8
S12342C0F5049093F7048093F6041092F5041092F404809184009091850090930B05809300
S12342E00A0510928500109284008091970590919805880F991F9093980580939705479A54
S12343001092E40580E09AEF90938B0080938A0080918A0090918B00909321068093200610
S123432080915406813021F080915406843011F481E013C080915406853021F08091540658
S1234340823011F482E009C080915406833021F080915406863029F483E080937606109276
S1234360E40586E990E0F0C08091F4049091F5049093F7048093F6041092F5041092F4043E
S1234380809184009091850090930B0580930A0510928500109284008091970590919805D1
S12343A0880F991F9093980580939705479A80918F05909190058051974208F0CAC08091C2
S12343C06A0690916B0685369105B4F11092E40580916A0690916B0690938B0080938A00F8
S12343E080918A0090918B00909321068093200680915406813021F080915406843011F49E
S123440081E013C080915406853021F080915406823011F482E009C080915406833021F0B7
S123442080915406863029F483E0809376061092E40584E090E088C080916A0690916B068E
S12344408B5B9F4FF4F11092E40584E690E090938B0080938A00909321068093200680915B
S12344605406813021F080915406843029F481E080937606459819C080915406853021F009
S123448080915406823029F482E08093760646980CC080915406833021F0809154068630F3
S12344A031F483E08093760644981092E40588E290E0909323068093220684E1809310058C
S12344C052C0809174069091750690938B0080938A00209125063091260680916A069091E9
S12344E06B06820F931F909321068093200680915406813021F080915406843029F481E0B7
S12345000E946B1981E019C080915406853021F080915406823029F482E00E946B1982E0E2
S12345200CC080915406833021F080915406863031F483E00E946B1983E08093E40584E1E9
S12345408093100584EB90E090932306809322060AC080912506909126068C509E4F90938A
S12345608B0080938A002B9A7894FF91EF91BF91AF919F918F917F916F915F914F913F919E
S12345802F910F900FBE0F901F9018951092800081EF9FEF909389008093880085EF9FEF87
S12345A090938B0080938A0080E88093810080EC9AED909385008093840083E090E0909388
S12345C00D0580930C0580910C0590910D0580688093810080916F00876080936F005398FC
S12345E052983D9A3E9A459A469A449AA2E0B2E00E943B2A802D8093F804A1E0B2E00E94F5
S12346003B2A802D8093F9048091F9048E3039F08091F904873119F087E18093F904809127
S1234620690084608093690080916900816080936900E99A089521EB30E0F901108210926C
S1234640B6001092B2001092B300A0E7B0E08C9183608C9338984098399841983A984298C3
S12346603B984398389839983A983B98EFE6F0E080818D7F80838C918C7F8C9386E0F901E6
S1234680808384E680931C060895813099F438983B9880912D01843021F439983A981092A9
S12346A012051092880610928706109211051092B1000895823049F439983A981092860618
S12346C0109285061092120515BC08951F920F920FB60F9211242F933F934F935F936F932B
S12346E07F938F939F93AF93BF93EF93FF93F89480911105843019F481E00E9445237894BD
S1234700FF91EF91BF91AF919F918F917F916F915F914F913F912F910F900FBE0F901F907B
S123472018950F931F9380912A0590912B050A9714F487E003C08091A10586E08093B1002F
S12347401092B20080918F0590919005845F914018F41092730616C080918F05909190059A
S12347608D56974020F08EE0809373060BC080918F059091900564E670E00E94D72965505A
S123478060937306E0917306F0E0E35DFC4F8081809313018091A105882329F02091F3011C
S12347A08091180108C0E0919305F0E0ED51FE4F808120911801829FC00111249093E905AC
S12347C08093E80580918F05909190058059914050F5809100019091010182FF1AC08091EA
S12347E0E8059091E90520911901820F911D9093E9058093E805809127069091280684602D
S1234800909328068093270680911A018093EA0541C080912706909128068B7F90932806EC
S12348208093270637C080912706909128068B7F90932806809327068091EA05823050F122
S12348408091EA0581508093EA05E091E805F091E905509119012091190180911A014091F1
S1234860EA0560911A01E50FF11D90E0841B910930E070E0AC01429FC001439F900D529F6F
S1234880900D11240E94D729E61BF70BF093E905E093E8058091A105882309F0E6C08091BA
S12348A07A0687FD3EC080917A068F30D4F5E0919305F0E0EC51FE4F6081E0919305F0E0BC
S12348C0ED51FE4F40810091E8051091E90580914E0620917A06E091180170E0641B710912
S12348E090E04AE0240290011124821B930B9C01629FC001639F900D729F900D11246AE0C8
S123490070E00E94EB29F0E06E9FC0016F9F900D7E9F900D1124800F911F9093E9058093F2
S1234920E8058091500687FD3EC0809150068930D4F5E0919305F0E0ED50FE4F6081E091FF
S12349409305F0E0ED51FE4F40810091E8051091E9058091770620915006E091180170E023
S1234960641B710990E04AE0240290011124821B930BAC01649FC001659F900D749F900DB7
S123498011246AE070E00E94EB29F0E06E9FC0016F9F900D7E9F900D1124800F911F9093F4
S12349A0E9058093E805809100019091010184FF5CC020915605309157058091360590919B
S12349C0370528173907FCF480913605909137052091560530915705821B930B64E070E087
S12349E00E94EB2980919405861710F460939405809194058A3018F089E080939405809194
S1234A0026018093EB053091EB053430C8F08091E8059091E905E0919405F0E0ED5DFC4F1F
S1234A202081820F911D9093E9058093E80531503093EB058091270690912806806109C016
S1234A40109294051092EB0580912706909128068F7E9093280680932706809136059091ED
S1234A6037059093570580935605809100019091010191FD09C08091280586FF94C0809155
S1234A80A105882309F48FC080911E068F5F80931E0690911E0680911F06981708F486C0AF
S1234AA010921E068091320590913305E0915006FF27E7FDF095E450FA4F208130E02817C8
S1234AC0390734F480911C0690911D06890F19C08091320590913305E0915006FF27E7FD10
S1234AE0F095E450FA4F208130E0821793075CF480911C0618163CF480911C0690911D0674
S1234B00891B80931C0680912706909128069D7F909328068093270620911C06E0915006E4
S1234B20FF27E7FDF095E450FA4F8089332727FD309590E08C599F4F8217930754F4E091EA
S1234B405006FF27E7FDF095E450FA4F80898C591EC020911C06E0915006FF27E7FDF095FA
S1234B60E450FA4F4089332727FD309584E690E0841B910928173907CCF4E0915006FF2769
S1234B80E7FDF095E450FA4F908984E6891B80931C068091270690912806926090932806FF
S1234BA08093270603C084E680931C068091E8059091E90520914D0630E062E070E00E94FA
S1234BC0EB29269FC001279F900D369F900D112464E670E00E94D729660F771F7093E905F5
S1234BE06093E805209140053091410580911C0190E0C296281739070CF04DC08091000144
S1234C009091010181FF47C08091400590914105C397D4F040911B0180911B0120914005FB
S1234C203091410560911C0190E070E06E5C7F4FFC01E29FC001E39F900DF29F900D112442
S1234C400E94D729461B03C080911B01482F50E08091E8059091E905480F591F5093E90509
S1234C604093E805189905C0809121019091220104C080911D0190911E01909320018093F9
S1234C801F0180912706909128068260909328068093270611C080912706909128068D7F86
S1234CA0909328068093270680911D0190911E019093200180931F018091F7059091F8054E
S1234CC083FF1CC0E091E805F091E90520913B018091E8059091E90564E170E00E94EB2960
S1234CE030E0629FC001639F900D729F900D11248E0F9F1F9093E9058093E80580910001DE
S1234D009091010190FF4CC080912A0590912B05823891050CF044C08091E8059091E905E3
S1234D2020912801820F911D9093E9058093E805E0912A05F0912B05609118012091280110
S1234D4082E890E08E1B9F0B70E0AB01849FB001859F700D949F700D11248FEF90E0FB01E2
S1234D60E89FB001E99F700DF89F700D1124882777FD8095982F30E040E050E00E94AC29D3
S1234D8020E43FE140E050E00E94FE298091E8059091E905820F931F9093E9058093E80571
S1234DA02091E8053091E9058091180145EF849FC00111248217930754F480911801849F63
S1234DC0C00111249093E9058093E8050BC08091E8059091E9051816190624F01092E905FF
S1234DE01092E8058091E8059091E905909396058093950578941F910F9108951F920F925D
S1234E000FB60F9211242F933F934F935F936F937F938F939F93AF93BF93EF93FF93F894EF
S1234E2020911105223039F0243009F44FC0213009F051C01CC080918706909188068F3F7A
S1234E409105D1F1C8F180918706909188068F5F8093B30080918706909188068F5F904031
S1234E6090938806809387062093110534C00E94912380919505909196059093880680939F
S1234E80870680918706909188068F3F9105A1F098F080918706909188068F5F8093B300B6
S1234EA080918706909188068F5F9040909388068093870682E007C080918706909188061C
S1234EC08093B30084E08093110505C081E00E944523109211057894FF91EF91BF91AF91E7
S1234EE09F918F917F916F915F914F913F912F910F900FBE0F901F9018951F920F920FB670
S1234F000F9211242F933F934F935F936F937F938F939F93AF93BF93EF93FF93F894209102
S1234F201205223039F0243009F453C0213009F053C020C080918506909186068F3F91058D
S1234F4091F088F080918506909186068F5F87BD80918506909186068F5F90409093860623
S1234F608093850633C0809185069091860687BD84E024C0809195059091960590938606B1
S1234F808093850624E025BD16BC80918506909186068F3F9105A9F0A0F080918506909124
S1234FA086068F5F87BD80918506909186068F5F9040909386068093850682E0809312054F
S1234FC00BC0809185069091860687BD2093120503C082E00E9445237894FF91EF91BF9110
S1234FE0AF919F918F917F916F915F914F913F912F910F900FBE0F901F9018951F920F92F4
S12350000FB60F9211242F933F934F935F936F937F938F939F93AF93BF93EF93FF93F894ED
S123502080911205843019F482E00E9445237894FF91EF91BF91AF919F918F917F916F910B
S12350405F914F913F912F910F900FBE0F901F90189554985C9855985D985498559815BC19
S1235060EEE6F0E080818360808384E085BD16BC82E187BD089511B88FEF84B915B887B954
S12350808AB90895089508950895089588E98093C10083E18093C40080ED96E090938E069E
S12350A080938D0690938A068093890680E996E090938C0680938B06909311078093100754
S12350C010928F061092240608951F920F920FB60F9211248F939F93EF93FF9380918F0631
S12350E0882311F1E0918D06F0918E0681918093C600F0938E06E0938D06E051F74030F056
S123510080ED96E090938E0680938D0680918F06815080938F0680918F06882329F48091AD
S1235120C1008F7D8093C100FF91EF919F918F910F900FBE0F901F9018951F920F920FB6EC
S12351400F9211242F938F939F93EF93FF938091C600E0911007F091110780838091240615
S12351608F5F80932406809110079091110701969093110780931007805D964030F080E967
S123518096E09093110780931007FF91EF919F918F912F910F900FBE0F901F901895809198
S12351A02406882319F48FEF9FEF0895F89480912406815080932406E0918B06F0918C0676
S12351C02191F0938C06E0938B06E05DF64030F080E996E090938C0680938B067894822F78
S12351E090E00895982F80918F068F33E0F780918F06803418F080E090E00895F89480912C
S12352008F068F5F80938F06E0918906F0918A0690838091890690918A06019690938A06A0
S1235220809389068051974030F080ED96E090938A06809389068091C10080628093C10040
S1235240789481E090E00895CF93DF93EC0104C00E94F2288111219688818823C9F781E071
S123526090E0DF91CF91089583E195E00E94242908958BE195E00E94242908958091240640
S123528090E00895CF92DF92EF92FF920F931F93CF93DF93CDB7DEB729970FB6F894DEBF2A
S12352A00FBECDBF8C01F62EE42EDE011196EEE1F5E089E001900D928150E1F749E06E01CA
S12352C00894C11CD11CFF2081F089E090E0841B91092F2D30E08217930738F04150F60173
S12352E0E40FF11D8CE28083FF244150F601E40FF11DC8016AE070E00E94D729805D8083A7
S1235300C8016AE070E00E94D7298B01672B11F4FF2019F085E08F15B0F619E01E197E01DB
S12353200894E11CF11C07C0F701E10FF11D80810E94F2281F5F1930B8F329960FB6F894C7
S1235340DEBF0FBECDBFDF91CF911F910F91FF90EF90DF90CF900895629FD001739FF001E5
S1235360829FE00DF11D649FE00DF11D929FF00D839FF00D749FF00D659FF00D9927729FE0
S1235380B00DE11DF91F639FB00DE11DF91FBD01CF0111240895991B79E004C0991F9617CB
S12353A008F0961B881F7A95C9F780950895AA1BBB1B51E107C0AA1FBB1FA617B70710F066
S12353C0A61BB70B881F991F5A95A9F780959095BC01CD01089597FB092E07260AD077FDB2
S12353E004D0E5DF06D000201AF4709561957F4F0895F6F7909581959F4F0895A1E21A2E29
S1235400AA1BBB1BFD010DC0AA1FBB1FEE1FFF1FA217B307E407F50720F0A21BB30BE40B80
S1235420F50B661F771F881F991F1A9469F760957095809590959B01AC01BD01CF01089538
S123544097FB092E05260ED057FD04D0D7DF0AD0001C38F450954095309521953F4F4F4F15
S12354605F4F0895F6F790958095709561957F4F8F4F9F4F0895F999FECFB2BDA1BDF89AC6
S1235480119600B40895F7DFE02DF5DFF02D0895F999FECFB2BDA1BD00BC11960FB6F894BF
S12354A0FA9AF99A0FBE0895F3DF012CF1DF11240895FFCF2F0001000200030004000500AA
S12354C00600070008003228E803900106141E1E3C581B581B88136419121E010102030412
S12354E00A0411C4098813C4096400DCE64003020A14324696500054819596B7AFC3C8BEBE
S1235500BEB9B0AFAFADAC4984C0CBD2D6D7D0C7C2BBB8B3AEAAA9458AA2A9AAB7C0BABE9F
S1235520BBB6B8B2B3B4B93281868DA4A58B8C8F9EA6A2A6A5A6C034525D5B596F7882859B
S1235540858281FF859FB034444E4B4A54615769727272737D9095272C1B252B334B5155CF
S1235560616A6D6C7D828B1D211A242A32454C4F5E6169717E81863432323232323232325F
S123558032327F3232323232323232323232323232323232323232131718191B1C1D1F214D
S12355A0232527282C2E311418191A1C2124272B3035393C3E414316191D232A31353B3F9E
S12355C042484E565A5E651B1D363E525863666C6E777D84898D932226434B6172818A901E
S12355E097A8ACAFB1B6B9292E484E6B7C939BA2AFB9BFCBD2D2D229344B536E7F9CA8B104
S1235600BCC5D0D2D2D2D2283F4E587187A4B2BAC2D2D2D2D2D2D23746545E7691B1BEC4C1
S1235620D2D2D2D2D2D2D239485660869FBAD2D2D2D2D2D2D2D2D200000000000000000030
S1235640000000000000000000000000000000000000000000000000000000000000000046
S12356600000000000000000000000000000000000000000000000010203040506070809F9
S12356800A0B0C0D0E0F100102030405060708090A0B0C0D0E0F10010203040506070809F6
S12356A00A0B0C0D0E0F1014161718191A1B1C1D1E1F2021222324191A1B1C1D1E1F2021BF
S12356C0222324252627271E1F2022232425262728292A2B2C2D2E000204060708090A0C25
S12356E00E28262422201E1E1E1E1E1E1E1E1E1E1EF0FF80BBE0880465484BA438022BF013
S1235700207019CC13860F440CC209D0074C061B052A046A03D1025602F201A1015F012821
S123572001FB00D600B7009D0087007500660059004D0044003C0034002E0029002500F017
S1235740FF80BBE0880465484BA438022BF0207019CC13860F440CC209D0074C061B052A03
S1235760046A03D1025602F201A1015F012801FB00D600B7009D0087007500660059004D3E
S12357800044003C0034002E0029002500F0FF80BBE0880465484BA438022BF0207019CCD9
S12357A013860F440CC209D0074C061B052A046A03D1025602F201A1015F012801FB00D624
S12357C000B7009D0087007500660059004D0044003C0034002E0029002500F0FF80BBE02F
S12357E0880465484BA438022BF0207019CC13860F440CC209D0074C061B052A046A03D13B
S1235800025602F201A1015F012801FB00D600B7009D0087007500660059004D0044003C5F
S12358200034002E00290025000000F5047E05AE066C08C00AB30D630F8B10D711881300F6
S12358400000000A000F001E003C007800FA007201E00180028002000008000A000C000EDB
S123586000C80A4A067E048403AC0D641A002000270032003E0066008E00B202EB0224034F
S123588037034B03560361037003E800D600C200B0009D008A00780078006500520040000E
S12358A02D001900070000000100010001175A5A5A505050505050505050505050506400FB
S11F58C0030000FA3204041B5B481B5B324A000D0A0020202020202020202000AA
S50302C733
